:1078000011E0A0E0B1E0E6ECFFE702C005900D92C8
:10781000A630B107D9F721E0A6E0B1E001C01D9282
:10782000AD34B207E1F7CDB7DEB72897DEBFCDBFE5
:10783000112484B78093270114BE88E180936000EF
:1078400089E280936000259A86E020E295B1922734
:1078500095B9E3EDF0E33197F1F700C000008150F6
:10786000A9F78091270181FF72C082E08093C00058
:1078700088E18093C10086E08093C2008CE0809311
:10788000C40010E000E0D12CC12CAA24AA94BA2C88
:1078900099249394A895F6D1813471F4F3D1F82EFC
:1078A0003AD3F2E8FF1202C083E004C021E885E683
:1078B000F212FACF29D304C0823421F484E137D301
:1078C000F12C40C0853411F485E0F9CF853541F4C1
:1078D000D9D1082FD7D1182F000F111F1CD3F0CFEB
:1078E000863521F484E023D380E0E4CF8436D9F4D4
:1078F000C9D1C8D1882EC6D1C80CD11CF12CF8141E
:1079000018F0C801CBD1EACFBDD1E82EBBD1F80128
:10791000EF0DF11D982F8E2D0C0197BEE8951124C7
:10792000F394F394ECCF843709F08BC0ABD1AAD198
:10793000F82EA8D1F0D2F80185918F01E5D2FA9402
:10794000F110F9CF80E1E0D2FF2009F4A3CF8EE25D
:1079500084B980E58CBD81E08DBD512C412C77240C
:107960007394AA24AA94BA2C8824839473E0972E43
:10797000EAE06E2EF999FECF43E050E070E060E05F
:1079800089E291E0FED248E050E06BE171E0CE0187
:107990000196F7D229982A9A63E083E2EBD161E05D
:1079A00085E2E8D167E286E2E5D163E780E5E2D1EE
:1079B00064E08DE3DFD161E082E2DCD161E081E26D
:1079C000D9D161E08CE3D6D121E041E070E060E004
:1079D00086E0A3D18732F9F480912A0180932801AF
:1079E0008FEF80932A0180932B018093080163E538
:1079F00084E2C0D143E26AE087E083D161E08EEFA8
:107A0000D8D1109208016FE584E2B4D180912A01A7
:107A10008F3F09F0A0C08D819E8124E0880F991FBF
:107A20002A95E1F74DD12F8138858217930709F008
:107A3000A1CF1CBCA89580912701282EF2010995A1
:107A400099CF853739F467D28EE15ED285E95CD271
:107A50008FE030CF813509F041CFBA82A982BC8254
:107A6000AB82C601F4E096958795FA95E1F79E837F
:107A70008D83C60125D198878F83CE0101965ED272
:107A80004AD2FF24F3945ECF870189819A81909333
:107A90000E0180930D018B819C8190931001809346
:107AA0000F01780181E0E81AF108F0921201E092EA
:107AB000110144EC62E382E024D163E083E079D1F8
:107AC000882309F46BC046E050E063E371E08DE089
:107AD00091E04AD2892BC9F6C8018150904F682F96
:107AE00062956077ACE2B1E0462F50E04C525140D5
:107AF000FA01EA0FFB1F1E963C911E971D962C91D2
:107B00001D97090177BEE89511241296E1E0AC3388
:107B1000BE0771F7611106C044E0880F991F4A95AE
:107B2000E1F7BCD0E114F10409F0AECFD886CF82E2
:107B30008D819E8134E0880F991F3A95E1F7C0D07E
:107B4000C816D90621F01E821D8218861F82CE011A
:107B50000196F4D10FCF8091290181508E3FF0F032
:107B600043E262E083E0CDD063E084E022D1882369
:107B700091F380912F01869586958695E3E3F1E058
:107B800060E0815020F490E080E00BD2F3CE919140
:107B9000669D900D1124692F6053F3CF70920D01F3
:107BA00010920E0143EC62E18FE0ABD060E08FE019
:107BB00000D18D819E8154E0880F991F5A95E1F77D
:107BC0007FD098878F8388E0FE013196ADE0B1E0E9
:107BD00001900D928A95E1F790921601809215011D
:107BE00044EC62E580E08DD063E081E0E2D0882360
:107BF00009F411CF48E050E063E371E0CE01019653
:107C0000B3D1892B09F407CF0091370110913801C6
:107C10000115110501F58091390190913A018A37DA
:107C20009A4DE9F4809133019091340181309105AE
:107C300051F46FEFC801B5D10F5F1F4F0115F4E08C
:107C40001F07B9F797CE02978230910508F092CEC0
:107C5000609135019ACF0038174008F0DCCE88E0FB
:107C6000E3E3F1E0DE01119601900D928A95E1F7D0
:107C7000CF80D884B886AF82CE0101965FD10D81C6
:107C80001E8103CF8091C00087FFFCCF8091C00090
:107C900084FD01C0A8958091C600089523E0FC01F1
:107CA00027BFE89507B600FCFDCF25E0FC0127BF04
:107CB000E89507B600FCFDCF81E187BFE895089500
:107CC000BC01F0E0E0E08FEF9FEFE617F70720F44C
:107CD000E11528E7F20708F008952591822748E08A
:107CE000DC01B695A7958170992722273327281B99
:107CF000390B2170307ACD0182279327415081F7CB
:107D0000E4CF90912901E6E0F1E0918390839FEF29
:107D1000968385834483638308952A9893E09A9594
:107D2000F1F700008EBD0DB407FEFDCF8EB59FEFBD
:107D3000415030F42A9AB3E0BA95F1F70000089563
:107D4000222369F09EBD0DB407FEFDCF8EB56115EF
:107D5000710571F3DB018C936F5F7F4FE9CFFB01FE
:107D60003196DB018C918EBD0DB407FEFDCF8EB533
:107D7000BF01DECFCF93DF931F92CDB7DEB769830C
:107D800020E041E0BE016F5F7F4FC7DF0F90DF91C2
:107D9000CF91089520E040E070E060E082EEBDDF2A
:107DA00020E040E070E060E081EEB7DF60E787E26E
:107DB000E1CFFF920F931F93CF93DF93C82FF62E3F
:107DC000D0910901D695D695D695D95F10912A0103
:107DD00029986EE080E2CEDF1093000120E045E0BC
:107DE00060E071E08AE299DF20E045E060E071E068
:107DF00080E393DF20E04D2F66E071E080EA8DDFC5
:107E0000299A00C000C020E040E070E060E08FEF01
:107E100084DF8073C1F32998BDDF6FE080E2AADFC1
:107E2000609129018AE2A6DF299A00E010E4A89572
:107E300021E041E070E060E087E16FDF80FF17C084
:107E40009FEF0150110919F0C913F1CF9C2FFA943B
:107E50008FEFF81619F0C913B3CF9C2F81E0C91327
:107E600080E0DF91CF911F910F91FF90089521E065
:107E700041E070E060E080E650DFD82F813208F00A
:107E8000D0E021E04D2F6CE271E081E646DF82DF39
:107E900080912F0186958695869590E00796D81754
:107EA000190671F690912E01809129019813C8CF7F
:107EB00090913101809130018770833009F0C1CFFA
:107EC000983009F0BECF8091280120912A01281313
:107ED00003C08F3F09F0B5CF20912D01821304C05C
:107EE00080932A019EEFADCF3091330181E0830F63
:107EF0008093330140912B01341708F0A2CF809377
:107F00002B0120932A019DCF9091C00095FFFCCFBB
:107F10008093C6000895B6DE803239F088E1809300
:107F2000600088E080936000FFCF84E1EDCFCF93C5
:107F3000C82FA8DEC150E9F7CF91EDCF0F931F9363
:107F4000CF93DF938C01CBE1D1E0F80161918F01F8
:107F5000CE0127D02196C332F1E0DF07B1F7DF91E0
:107F6000CF911F910F910895FB01DC0104C08D9109
:107F70000190801921F441505040C8F7881B990B9B
:107F80000895DC01CB01FC01F999FECF06C0F2BDDA
:107F9000E1BDF89A319600B40D9241505040B8F7C7
:107FA0000895262FF999FECF92BD81BDF89A0197C9
:107FB00000B4021639F01FBA20BD0FB6F894FA9A31
:067FC000F99A0FBE0895BE
:067FC60000FCE1A8A80088
:107FCC00040000001400000003000000474E5500A0
:107FDC001F7404E583E90C8D5085405A2D9E08FCD6
:047FEC008D5E22FC88
:040000030000780081
:00000001FF
